:0400000057EF00F0C6
:100008000548054805480548054805480548054880
:100018000548054805480548054805480548054870
:100028000548054805480548054805480548054860
:10003800054805480548EF45054805480548054869
:1000480005480548054805482B0005480548054862
:100058000548054805480548054805480548054830
:100068000548054805480548054805480548054820
:10007800054805482B000548054805482B002B0076
:100088002B002B002B002B002B002B0005480548CC
:10009800BF460548054805482B002B002B002B00C0
:0A00A80005480548FF0089EF8BF0C2
:10FCE0000001020408102040804C4C4C48004C4C51
:10FCF000484C004C4C48480048484C48004C484C44
:10FD00004C004C484C48004C48484C004848484C33
:10FD1000004C48484800484C4C4C00484C4C48006B
:10FD20004848484800484C484C00484C484800481F
:10FD3000484C4C004C4C4C4C002050726F6A65741F
:10FD4000204D504C414258203A2047656E65726103
:10FD5000746575725F44544D465F31384632374B97
:10FD600034325F323032322028706F757220506F1B
:10FD7000727469657220417564696F70686F6E6531
:10FD8000290D0A0020436F6D70696C65206C652039
:10FD900025732061202573205554430D0A20617678
:10FDA00065632076657273696F6E20584338203A18
:10FDB00020202564206574205041434B2025730D7D
:10FDC0000A00204C6564733A2025732020546F7517
:10FDD0006368653D202563202020523D2563202057
:10FDE000433D2563202046313D25356420487A2057
:10FDF000202046323D25356420487A0D0A002048EF
:10FE000061726477617265203A2050494331384607
:10FE100032374B3432202C20464F534320696E74C6
:10FE200065726E65203D36344D487A200D0A0020FB
:10FE300055736167652064652054696D6572312072
:10FE40007820666F6973203130306D53202C205438
:10FE5000696D65723420203130306D530D0A0020F9
:10FE6000496E697420505752352028736F72746937
:10FE7000652072E92D61696775696C6CE9652073AD
:10FE8000757220524334290D0A0020526F77203AB0
:10FE900020202036393720202020373730202020DE
:10FEA0002038353220202020393431202020204FA6
:10FEB00046460D0A0020436F6C203A202031323034
:10FEC0003920202031333336202020313437372079
:10FED000202031363333202020204F46460D0A00A3
:10FEE00020496E69742054696D65723220617373A4
:10FEF0006F6369E920E02050574D35202C2074694C
:10FF0000636B3D3634B5530D0A0020496E69742089
:10FF1000657420746573742054696D657236202D84
:10FF20003E20382078203530306D53203A20002094
:10FF3000554152543120205243363D5458202031EF
:10FF400031353230302C382C4E2C31200D0A002027
:10FF500053696E65776176652044544D4620676528
:10FF60006E657261746F720D0A002053656C656373
:10FF7000742074686520322044544D4620746F6E9E
:10FF800065730D0A002056657273696F6E203A2002
:10FF9000323032322D313230360D0A005049433181
:10FFA00038462D4B5F44465020312E362E313235A7
:10FFB0000020436F6E6669673D20484F4D450D0A2E
:10FFC000002044757479203D20253564200D0A00F9
:10FFD0004465632020362032303232006364653D50
:10FFE000527843780D0A00205465737420555020D0
:0FFFF0000031363A30353A3335006C6C7300000F
:020000040001F9
:10000000FDEC8FF00D0E3A01146F000E126F1CEC18
:100010008FF0000E0101ED6F7F0EEC6F000E0001FE
:10002000B56F000EB46F1FEF80F0000EB425D96ECF
:10003000010EB521DA6E000EDF6EB44BB52B010157
:10004000EC510001B45D0101ED510001B559D8A09A
:100050002CEF80F02EEF80F015EF80F0000EB56FE2
:10006000000EB46F000EB425D96E020EB521DA6E03
:10007000000EDF6EB44BB52BB55109E14F0EB45DE8
:10008000D8A045EF80F047EF80F032EF80F0000E0F
:10009000B56F000EB46F000EB425D96E030EB521F6
:1000A000DA6E000EDF6EB44BB52BB55109E17F0E51
:1000B000B45DD8A05EEF80F060EF80F04BEF80F091
:1000C000000EA46F030EA56F76EC8EF0000E0001FB
:1000D000A46F030EA56F600093F2D9FF600097F242
:1000E000DAFF000EDF6E72EC8FF0000E0001956FEC
:1000F000000E946F000E916F000E906F000E8F6FC8
:100100000A0E8E6F000E8B6F000E8A6F000E816FCD
:10011000000E806F000E7F6F000E7E6F72EC8FF00E
:10012000390E2C6EFD0E2D6ED7EC8DF0850E2C6EDB
:10013000FF0E2D6ED7EC8DF0A4C0DBF0A5C0DCF077
:10014000840E0001DD6FFD0EDE6FD00EDF6FFF0E3F
:10015000E06FF10EE16FFF0EE26F090EE46F380EF3
:10016000E36F9C0EE56FFF0EE66F1EEC8DF0DBC0BB
:10017000ECF1DCC0EDF1A4C02CF0A5C02DF0B1EC89
:100180008CF0FE0E2C6EFD0E2D6ED7EC8DF02F0E2A
:100190002C6EFF0E2D6ED7EC8DF02F0E2C6EFE0EFA
:1001A0002D6ED7EC8DF0B10E2C6EFF0E2D6ED7ECB0
:1001B0008DF072EC8FF0D28E5F0E2C6EFE0E2D6ED7
:1001C000D7EC8DF0F1EC8FF0E00E2C6EFE0E2D6E64
:1001D000D7EC8DF0AC8EE70E2C6EFF0E2D6ED7ECAB
:1001E0008DF0000E0001B76F800EB66FA4C0DBF07B
:1001F000A5C0DCF0C10EDD6FFF0EDE6FB6C0DFF014
:10020000B7C0E0F01EEC8DF0A4C02CF0A5C02DF01E
:10021000B1EC8CF0BA84B6C02CF0B7C02DF058EC1D
:100220008FF0BA94CCEC8FF0800E0001B625B66F3B
:10023000000EB721B76F810EB65D030EB759D8A077
:1002400024EF81F026EF81F0F6EF80F00A0E2C6E9D
:10025000FF0E2D6ED7EC8DF0080E4FEC8DF03901AE
:100260009981D28E43EF81F02E0EBFEC8FF0290ED4
:100270000001FB6F960EFA6F7F0EE82EFED7FA2F65
:10028000FCD7FB2FFAD70001BFAB49EF81F04BEF52
:1002900081F034EF81F072EC8FF072EC8FF04F0E42
:1002A0002C6EFF0E2D6ED7EC8DF06A0E2C6EFF0EAD
:1002B0002D6ED7EC8DF08A0E2C6EFE0E2D6ED7ECC7
:1002C0008DF0B50E2C6EFE0E2D6ED7EC8DF072EC0F
:1002D0008FF0D28E000E0001B56F000EB46F000ECD
:1002E000836F000E826F000ECD6F000ECC6F2CEC72
:1002F0008CF0A30E0001FB6F570EFA6F020EE82E72
:10030000FED7FA2FFCD7FB2FFAD700F00001C40567
:10031000D8A48DEF81F08FEF81F0E1EF81F0520EE4
:1003200001010019D8A497EF81F099EF81F0E1EF76
:1003300081F0430E0219D8A4A0EF81F0A2EF81F062
:10034000E1EF81F0000E2C6E020E2D6EDC0E2E6E93
:10035000FF0E2F6E2BEC8EF001C1C7F02F0E0001A7
:10036000C765B5EF81F0B7EF81F0C4EF81F0340ECF
:10037000C761BDEF81F0BFEF81F0C4EF81F0C7C06E
:1003800005F2C751D00FCD6F03C1C7F02F0EC7655F
:10039000CCEF81F0CEEF81F0DBEF81F0340EC7615E
:1003A000D4EF81F0D6EF81F0DBEF81F0C7C007F228
:1003B000C751D00FCC6F000E2C6E020E2D6EB1EC1B
:1003C0008CF00001CD51FA6FFB6BD890FA37FB37F8
:1003D000D890FA37FB37CC51FA25B46F000EFB21C9
:1003E000B56FB4C02CF0B5C02DF0000E2F6E050E09
:1003F0002E6E89EC8FF0E90E2C240001FD6FFC0EAF
:100400002D20FE6FA4C0DBF0A5C0DCF0C20EDD6FB6
:10041000FD0EDE6FFDC0DFF0FEC0E0F0A40EB425DF
:10042000D96E010EB521DA6EDF50FA6FFA51E16F25
:10043000E26B300ECD25E36FE46B000EE423300E4B
:10044000CC25E56FE66B000EE623CD51020DDD0EE7
:10045000F324D96E010EF420DA6E6F0078FFE7F016
:100460006F0074FFE8F0CC51020DD50EF324D96E65
:10047000010EF420DA6E6F0078FFE9F06F0074FF70
:10048000EAF01EEC8DF0A4C02CF0A5C02DF0B1EC6C
:100490008CF00001CD51040DC50EF324D96E010E70
:1004A000F420DA6E6F0078FF28F06F0078FF29F0F3
:1004B0006F0078FF2AF06F0078FF2BF0CC51040D0D
:1004C000B50EF324D96E010EF420DA6E6F0078FFBA
:1004D000C6F26F0078FFC7F26F0078FFC8F26F00B6
:1004E00078FFC9F2000E4FEC8DF0CBEF82F0A4A59F
:1004F0007CEF82F07EEF82F077EF82F0A4956E8E33
:1005000028502024206E29502120216E2A5022209C
:10051000226E2B502320236E22503F0B0001FA6FD6
:10052000FB6B500EFA25D96E020EFB21DA6EDF50FE
:10053000FC6FFC51B66FB76B0201C6512424246EC8
:10054000C7512520256EC8512620266EC951272067
:10055000276E26503F0B0001FA6FFB6B800EFA25C9
:10056000D96E030EFB21DA6EDF50FC6FFC51B6250D
:10057000B66F000EB721B76FD890B635B66FB735E6
:10058000B76F800EB627000EB723B6C02CF0B7C0E9
:100590002DF058EC8FF03901A9A1D1EF82F0D3EF03
:1005A00082F077EF82F06E9E77EF81F057EF00F0E8
:1005B00060006FF1D9FF600073F1DAFF6F007BFF1D
:1005C000F6FF6F0077FFF7FF000EF86E0800F5509A
:1005D000250AD8A4EEEF82F0F0EF82F025EF85F047
:1005E00060006FF1D9FF600073F1DAFFDE2A000EC0
:1005F000DD22000E0001776F000E766F76C07AF074
:1006000077C07BF07869796960006FF1D9FF60008D
:1006100073F1DAFF6F007BFFF6FF6F0077FFF7FFE4
:10062000000EF86E0800F5502A0AD8A41AEF83F0DD
:100630001CEF83F04FEF83F060006FF1D9FF600093
:1006400073F1DAFFDE2A000EDD22600077F1D9FFB8
:1006500060007BF1DAFF6F007CFF13F0020EDE26F4
:100660006F007CFF14F0000EDD2260004FF0D9FF18
:10067000600053F0DAFF6F0078FF76F06F0074FFD0
:1006800077F077BF48EF83F046EF83F091EF83F088
:100690007A81766D771FD8B0772B91EF83F0600069
:1006A0006FF1D9FF600073F1DAFF6F0078FF33F06C
:1006B0006F0074FF34F054EC88F033C076F034C02F
:1006C00077F06CEF83F060006FF1D9FF600073F199
:1006D000DAFFDE2A000EDD22D00E136EFF0E146E3E
:1006E00060006FF1D9FF600073F1DAFF6F007BFFEC
:1006F000F6FF6F0077FFF7FF000EF86E0800F55069
:10070000156E166A1350152614501622165009E15C
:100710000A0E155CD8A08FEF83F091EF83F063EFA2
:1007200083F060006FF1D9FF600073F1DAFF6F00B2
:100730007BFFF6FF6F0077FFF7FF000EF86E0800F3
:10074000F550630AD8A4A7EF83F0A9EF83F0D9EF9F
:1007500083F060006FF1D9FF600073F1DAFFDE2AE9
:10076000000EDD22600077F1D9FF60007BF1DAFF37
:100770006F007CFF13F0020EDE266F007CFF14F08A
:10078000000EDD2260004FF0D9FF600053F0DAFF69
:10079000DF500001DA6F59C035F05AC036F0DAC0C8
:1007A00037F04EEC8AF035C059F036C05AF048EFB9
:1007B00085F060006FF1D9FF600073F1DAFF6F0020
:1007C0007BFFF6FF6F0077FFF7FF000EF86E080063
:1007D000F550640AD8B4EFEF83F0F1EF83F009EF3E
:1007E00084F060006FF1D9FF600073F1DAFF6F00F1
:1007F0007BFFF6FF6F0077FFF7FF000EF86E080033
:10080000F550690AD8A407EF84F009EF84F054EF9B
:1008100084F060006FF1D9FF600073F1DAFFDE2A27
:10082000000EDD22600077F1D9FF60007BF1DAFF76
:100830006F007CFF13F0020EDE266F007CFF14F0C9
:10084000000EDD2260004FF0D9FF600053F0DAFFA8
:100850006F0078FFCEF06F0074FFCFF00001000E44
:10086000CFBFFF0ED06FD16FD26FD36FD46FD56F64
:1008700059C047F05AC048F0CEC049F0CFC04AF046
:10088000D0C04BF0D1C04CF0D2C04DF0D3C04EF030
:10089000D4C04FF0D5C050F049EC85F047C059F0B6
:1008A00048C05AF048EF85F060006FF1D9FF600052
:1008B00073F1DAFF6F007BFFF6FF6F0077FFF7FF42
:1008C000000EF86E0800F550730AD8B46AEF84F091
:1008D0006CEF84F08BEF84F060006FF1D9FF600063
:1008E00073F1DAFF6F0078FF2CF06F0074FF2DF0CA
:1008F000FA0E2E6EFF0E2F6E000E316E030E306E4E
:10090000C5EC89F02C502D10D8A489EF84F08BEF22
:1009100084F0E5EF84F060006FF1D9FF600073F1BF
:10092000DAFF6F007BFFF6FF6F0077FFF7FF000E27
:10093000F86E0800F550730AD8B4A1EF84F0A3EF65
:1009400084F0AAEF84F0000E0001D96F030ED86F77
:10095000AFEF84F0000E0001D96F010ED86F600078
:100960006FF1D9FF600073F1DAFFD851DE26D9515B
:10097000DD22600077F1D9FF60007BF1DAFF6F00C4
:100980007CFF13F0020EDE266F007CFF14F0000ED9
:10099000DD2260004FF0D9FF600053F0DAFF6F00F6
:1009A00078FFD6F06F0074FFD7F059C035F05AC009
:1009B00036F0D6C037F0D7C038F0BCEC86F035C082
:1009C00059F036C05AF048EF85F060006FF1D9FF5A
:1009D000600073F1DAFF6F007BFFF6FF6F0077FFB7
:1009E000F7FF000EF86E0800F550250AD8A4FBEFBB
:1009F00084F0FDEF84F016EF85F060006FF1D9FF11
:100A0000600073F1DAFFDE2A000EDD22000E2D6E8B
:100A1000250E2C6E59C02EF05AC02FF0BAEC8AF079
:100A2000000E5A6E010E596E48EF85F060006FF1AE
:100A3000D9FF600073F1DAFFDE2A000EDD22000E1E
:100A40005A6E000E596E48EF85F060006FF1D9FFC5
:100A5000600073F1DAFF6F007BFFF6FF6F0077FF36
:100A6000F7FF000EF86E0800F5502C6E2D6A59C085
:100A70002EF05AC02FF0BAEC8AF060006FF1D9FF67
:100A8000600073F1DAFFDE2A000EDD2210EF85F040
:100A9000120049C009F04AC00AF04BC00BF04CC02C
:100AA0000CF04DC00DF04EC00EF04FC00FF050C016
:100AB00010F010BE5EEF85F061EF85F0010E62EF81
:100AC00085F0000E076E086A07500810D8B46BEF67
:100AD00085F06DEF85F07DEF85F0101E0F1E0E1E68
:100AE0000D1E0C1E0B1E0A1E096C000E0A220B2284
:100AF0000C220D220E220F221022000179BF83EF5B
:100B000085F085EF85F086EF85F07A9379BF93EFD6
:100B100085F0795106E17805D8B091EF85F093EF33
:100B200085F099EF85F0000E046E010E036E9DEFC7
:100B300085F078C003F079C004F076C005F077C086
:100B400006F007500810D8A4A8EF85F0AAEF85F0AA
:100B5000B1EF85F07AA5AFEF85F0B1EF85F0B4EF96
:100B600085F00506D8A00606000E126E1F0E116E47
:100B7000000E0101A36F39EF86F01106D8A012060E
:100B8000840E1124D96E010E1220DA6E09C02CF0E9
:100B90000AC02DF00BC02EF00CC02FF00DC030F0AD
:100BA0000EC031F00FC032F010C033F00A0E346EB8
:100BB000000E356E000E366E000E376E000E386E6B
:100BC000000E396E000E3A6E000E3B6E13EC89F08B
:100BD0002CC051F02DC052F02EC053F02FC054F055
:100BE00030C055F031C056F032C057F033C058F025
:100BF00051C03EF053C03FF0FCEC8EF03E50300F41
:100C0000DF6E0306D8A004060506D8A0060609C0B4
:100C10002CF00AC02DF00BC02EF00CC02FF00DC030
:100C200030F00EC031F00FC032F010C033F00A0EB9
:100C3000346E000E356E000E366E000E376E000EEE
:100C4000386E000E396E000E3A6E000E3B6E90EC60
:100C500087F02CC009F02DC00AF02EC00BF02FC079
:100C60000CF030C00DF031C00EF032C00FF033C0C8
:100C700010F012BE44EF86F0125008E11104D8A023
:100C800044EF86F046EF86F077EF86F009500A10C1
:100C90000B100C100D100E100F101010D8A453EFE5
:100CA00086F055EF86F0BDEF85F004BE62EF86F06A
:100CB000045006E10304D8B060EF86F062EF86F0DE
:100CC000BDEF85F006BE6DEF86F0065008E1050425
:100CD000D8A06DEF86F06FEF86F077EF86F0000119
:100CE0007AB375EF86F077EF86F0BDEF85F00750A9
:100CF0000810D8A47EEF86F080EF86F088EF86F0AB
:100D000000017AA586EF86F088EF86F0A7EF86F0DF
:100D10001106D8A0120607500810D8A492EF86F04A
:100D200094EF86F09AEF86F0000E026E2B0E016EA5
:100D30009EEF86F0000E026E2D0E016E840E1124C1
:100D4000D96E010E1220DA6E600007F0DFFF47C097
:100D50003CF048C03DF0840E11243E6E010E12207E
:100D60003F6E05C040F006C041F026EC8BF03CC061
:100D700047F03DC048F0120020EEE5F110EE3AF0E9
:100D8000060E6F006FFFE3FFE806FBE237C045F099
:100D900038C046F045504610D8A4D1EF86F0D3EFC6
:100DA00086F0D7EF86F03A0E456E000E466E45C0CF
:100DB0002CF046C02DF0ABEC8DF02CC049F02DC0CE
:100DC0004AF078C047F079C048F048BEEAEF86F0B4
:100DD000ECEF86F001EF87F04950475C4850800AFD
:100DE000396E4A50800A3958D8A0F9EF86F0FBEFE7
:100DF00086F0FDEF86F001EF87F047C049F048C06C
:100E00004AF049C047F04AC048F076C043F077C086
:100E100044F000017AB10FEF87F011EF87F02EEF69
:100E200087F01FEF87F0000E2D6E200E2C6E35C060
:100E30002EF036C02FF0BAEC8AF0494A4A2A4350C5
:100E4000495C4A50800A396E4450800A3958D8A00B
:100E50002CEF87F02EEF87F013EF87F0000E426E35
:100E6000000E416E57EF87F0600017F1F6FF60004B
:100E70001BF1F7FF000EF86E1F0EF76403D0080099
:100E8000F55007D06F00DBFFE1FF6F00DFFFE2FFEF
:100E9000E750396E39502C6E2D6A35C02EF036C0B1
:100EA0002FF0BAEC8AF0454A462A414A422A475076
:100EB000415C4250800A396E4850800A3958D8A0A7
:100EC00064EF87F066EF87F034EF87F000017AA1D6
:100ED0006CEF87F06EEF87F08BEF87F07CEF87F099
:100EE000000E2D6E200E2C6E35C02EF036C02FF069
:100EF000BAEC8AF0494A4A2A4350495C4A50800A6F
:100F0000396E4450800A3958D8A089EF87F08BEFAA
:100F100087F070EF87F049C035F04AC036F0120014
:100F2000000E3D6E3BBE99EF87F097EF87F0ABEF79
:100F300087F03B1E3A1E391E381E371E361E351EE0
:100F4000346C000E352236223722382239223A22DA
:100F50003B22010E3D6E33BEB2EF87F0B0EF87F05B
:100F6000C4EF87F0331E321E311E301E2F1E2E1E80
:100F70002D1E2C6C000E2D222E222F2230223122EB
:100F800032223322010E3D1A20EE3EF0070EDE6AB9
:100F9000E806FDE23450351036103710381039109D
:100FA0003A103B10D8B4D7EF87F0D9EF87F02BEF8A
:100FB00088F0010E3C6EE7EF87F0D8903436353676
:100FC00036363736383639363A363B363C2A3BAE3B
:100FD000ECEF87F0EEEF87F0DDEF87F0D8903E364C
:100FE0003F36403641364236433644364536345035
:100FF0002C5C35502D5836502E5837502F583850BD
:101000003058395031583A5032583B503358D8A0A4
:101010000CEF88F00EEF88F01FEF88F034502C5E54
:1010200035502D5A36502E5A37502F5A3850305A84
:101030003950315A3A50325A3B50335A3E80D89048
:101040003B323A3239323832373236323532343254
:101050003C2EEEEF87F03D50D8B431EF88F033EFFF
:1010600088F043EF88F0451E441E431E421E411E79
:10107000401E3F1E3E6C000E3F2240224122422273
:101080004322442245223EC02CF03FC02DF040C0F8
:101090002EF041C02FF042C030F043C031F044C0C8
:1010A00032F045C033F01200000E3C6E000E3B6E75
:1010B000000E3A6E000E396E60EF88F0334A342A23
:1010C0006000CFF0F6FF6000D3F0F7FF000EF86E7F
:1010D0000800F550200AD8B470EF88F072EF88F05D
:1010E0005EEF88F0F70E356EFF0E366E6000CFF0C3
:1010F000F6FF6000D3F0F7FF000EF86E0800F55021
:10110000376E386A3550372636503822385009E164
:10111000050E375CD8A08FEF88F091EF88F05EEF76
:1011200088F09BEF88F0000E3A6E010E396E334A5C
:10113000342AD8EF88F06000CFF0F6FF6000D3F0DB
:10114000F7FF000EF86E0800F550356E366A36501F
:10115000000AD8B4AEEF88F0D8EF88F035502B0AEB
:10116000D8B497EF88F0060AD8B493EF88F0D8EF98
:1011700088F03BC02CF03CC02DF0000E2F6E0A0E04
:101180002E6E89EC8FF06000CFF0F6FF6000D3F098
:10119000F7FF000EF86E0800F5502C5E000E2D5A79
:1011A000300E2C243B6E000E2D203C6E97EF88F005
:1011B000D00E356EFF0E366E6000CFF0F6FF600089
:1011C000D3F0F7FF000EF86E0800F550376E386A5E
:1011D0003550372636503822385009E10A0E375C30
:1011E000D8A0F5EF88F0F7EF88F0B9EF88F0395024
:1011F0003A10D8A4FEEF88F000EF89F00EEF89F0E6
:101200003BC035F03CC036F0351E361E354A362A16
:1012100035C033F036C034F012EF89F03BC033F004
:101220003CC034F01200000E3D6E33BE1CEF89F05E
:101230001AEF89F02EEF89F0331E321E311E301E58
:101240002F1E2E1E2D1E2C6C000E2D222E222F2224
:101250003022312232223322010E3D6E3BBE35EF69
:1012600089F033EF89F045EF89F03B1E3A1E391EB5
:10127000381E371E361E351E346C000E35223622BF
:101280003722382239223A223B2234503510361088
:101290003710381039103A103B10D8B452EF89F09B
:1012A00054EF89F09CEF89F0010E3C6E62EF89F0FB
:1012B000D8903436353636363736383639363A36CB
:1012C0003B363C2A3BAE67EF89F069EF89F058EF77
:1012D00089F034502C5C35502D5836502E583750EC
:1012E0002F5838503058395031583A5032583B50B6
:1012F0003358D8A07EEF89F080EF89F090EF89F025
:1013000034502C5E35502D5A36502E5A37502F5AA5
:101310003850305A3950315A3A50325A3B50335A79
:10132000D8903B323A32393238323732363235326F
:1013300034323C2E69EF89F03D50D8B4A2EF89F0E9
:10134000A4EF89F0B4EF89F0331E321E311E301E37
:101350002F1E2E1E2D1E2C6C000E2D222E222F2213
:1013600030223122322233222CC02CF02DC02DF01D
:101370002EC02EF02FC02FF030C030F031C031F031
:1013800032C032F033C033F012002CC033F02DC025
:1013900034F02EC035F02FC036F03006D8A031061C
:1013A000302806E13128D8A4D8EF89F0DAEF89F0A7
:1013B000E7EF89F0000E2D6E000E2C6E4DEF8AF0D7
:1013C000334A342A354A362A3006D8A0310660001E
:1013D000CFF0F6FF6000D3F0F7FF000EF86E0800C4
:1013E000F5500009D8B4F7EF89F0F9EF89F032EF42
:1013F0008AF06000D7F0F6FF6000DBF0F7FF000E28
:10140000F86E0800F5500009D8B409EF8AF00BEF28
:101410008AF032EF8AF030503110D8B412EF8AF0EF
:1014200014EF8AF032EF8AF06000CFF0F6FF600030
:10143000D3F0F7FF000EF86E08006F00D4FF32F013
:101440006000D7F0F6FF6000DBF0F7FF000EF86EEB
:101450000800F5503218D8B430EF8AF032EF8AF035
:10146000E0EF89F06000CFF0F6FF6000D3F0F7FF07
:10147000000EF86E08006F00D4FF32F06000D7F065
:10148000F6FF6000DBF0F7FF000EF86E0800F55085
:10149000325C2C6E2D6AD8A02D0612000001765108
:1014A0007711D8A456EF8AF058EF8AF05EEF8AF0F1
:1014B00076C03BF077C03CF064EF8AF0FF0E7625F3
:1014C0003B6EFF0E77213C6E7AA169EF8AF06BEFDD
:1014D0008AF074EF8AF037C02CF02D6A35C02EF0F8
:1014E00036C02FF0BAEC8AF03CBE79EF8AF07BEF81
:1014F0008AF07DEF8AF081EF8AF0000E3C6E000EDC
:101500003B6E000E3A6E000E396E93EF8AF0000EBD
:101510002D6E200E2C6E35C02EF036C02FF0BAEC9A
:101520008AF0394A3A2A3B50395C3A50800A386E80
:101530003C50800A3858D8A0A0EF8AF0A2EF8AF079
:1015400087EF8AF000017AB1A8EF8AF0AAEF8AF05B
:10155000B3EF8AF037C02CF02D6A35C02EF036C0BC
:101560002FF0BAEC8AF0010E3924356E000E3A20C5
:10157000366E12002E502F10D8B4C1EF8AF0C3EF90
:101580008AF0CCEF8AF02E502F10D8A4CAEF8AF040
:10159000CCEF8AF0D1EF8AF02C5008EC90F025EFD8
:1015A0008BF020EE09F02E50D9262F50DA22DE5093
:1015B000DE10D8B4DEEF8AF0E0EF8AF0FBEF8AF0BD
:1015C00020EE09F02E50D9262F50DA2210EE03F02B
:1015D0002E50E1262F50E222DE50E65CE650800AD3
:1015E000346EDE50800A3458D8B0F9EF8AF0FBEF41
:1015F0008AF025EF8BF020EE03F02E50D9262F50E5
:10160000DA226F0078FF30F06F0074FF31F0600075
:10161000BBF0D9FF6000BFF0DAFF6F0078FF32F057
:101620006F0074FF33F030503224D96E31503320C4
:10163000DA6E6000B3F0DFFF20EE03F02E50D92603
:101640002F50DA22DE2A000EDD22120000017AA1DC
:101650002CEF8BF02EEF8BF038EF8BF03EC035F097
:101660003FC036F03CC037F03DC038F09AEC8EF009
:1016700041BE3DEF8BF03FEF8BF045EF8BF040C06C
:1016800045F041C046F049EF8BF0000E466E000E6B
:10169000456E000E446E000E436E5BEF8BF0000E45
:1016A0002D6E200E2C6E3CC02EF03DC02FF0BAECFB
:1016B0008AF0434A442A4550435C4450800A426EB3
:1016C0004650800A4258D8A068EF8BF06AEF8BF042
:1016D0004FEF8BF000017AB170EF8BF072EF8BF06F
:1016E0007CEF8BF03EC035F03FC036F03CC037F0A9
:1016F0003DC038F09AEC8EF03EC02CF03FC02DF08B
:10170000ABEC8DF045502C243C6E46502D203D6EA8
:101710001200B80EF66E1D0EF76E010EF86E00EE9A
:1017200080F310EE40F009006F00D7FFEEFFE550A8
:10173000E150F9E1A40EF66E1C0EF76E010EF86E84
:1017400000EEA4F110EE48F009006F00D7FFEEFFA5
:10175000E550E150F9E1780EF66E1D0EF76E010EC0
:10176000F86E00EE50F210EE40F009006F00D7FF67
:10177000EEFFE550E150F9E100EE00F3800EEE6A75
:10178000E806FDE100EE00F1A40EEE6AE806FDE1D8
:1017900000EE00F2500EEE6AE806FDE100EE60F0A9
:1017A0006E0EEE6AE806FDE15F6A080ED56E000E69
:1017B000D66E000ED76E000100EF80F03901A3A7AE
:1017C000E4EF8BF0E6EF8BF02BEF8CF093A7EBEFD1
:1017D0008BF0EDEF8BF02BEF8CF06F00A0F75FF04C
:1017E0000D0E5F18D8B4F7EF8BF0F9EF8BF005EF23
:1017F0008CF00001A75109E1800EA65DD8A003EF8F
:101800008CF005EF8CF01CEF8CF0010E0001C46F22
:10181000000EA625D96E010EA721DA6E000EDF6E2E
:10182000A6C0A8F0A7C0A9F0000EA76F000EA66F73
:10183000390193972BEF8CF0000EA625D96E010E7F
:10184000A721DA6E60007FF1DFFFA64BA72BA6C0B1
:10185000A8F0A7C0A9F011003901A3A732EF8CF0BE
:1018600034EF8CF037EF8CF06F00A0F75FF0000ED4
:101870000001A76F000EA66FA75109E17F0EA65DBC
:10188000D8A045EF8CF047EF8CF049EF8CF05EEF7D
:101890008CF0000EA625D96E010EA721DA6E000E7F
:1018A000DF6EA64BA72BA75109E17F0EA65DD8A03E
:1018B0005CEF8CF05EEF8CF049EF8CF0000EC46FA3
:1018C0003D01F289000EF96F000EFA6F000E010162
:1018D000006F000E0001A76F000EA66F000EA96F2B
:1018E000000EA86F000E5F6E3901938D9387120072
:1018F000000EBA6E000EBB6E000EBC6E010EC26E04
:10190000C3688F0EC46E000E3A01606FC00E506F38
:10191000000E406F000E816F000E516F000E416F80
:10192000800E616F000E5A6F000E5B6F000E6A6FC3
:10193000000E6B6F000E426F000E526F000E626F52
:10194000436953696369446954696469080E846F23
:10195000090E146F000E126F130E166F170EE56F3F
:101960001200000E00017D6F000E7C6FDAEF8CF02C
:101970003901A3A9BEEF8CF0C0EF8CF0B8EF8CF06A
:1019800000017C512C24D96E7D512D20DA6EDF5060
:101990003D01EA6F00017C4B7D2B7D5109E1810EF9
:1019A0007C5DD8A0D6EF8CF0D8EF8CF0DAEF8CF01D
:1019B000E8EF8CF07C512C24D96E7D512D20DA6E0D
:1019C000DF50D8A4E6EF8CF0E8EF8CF0B8EF8CF0A5
:1019D000120019C01DF01AC01EF0000E0001756F34
:1019E000000E746F07EF8DF017C059F018C05AF051
:1019F0001D0E5B6E000E5C6E1BC05DF01CC05EF0C9
:101A0000D8EC82F05950000174275A5075236000B9
:101A100077F0F6FF60007BF0F7FF000EF86E08002D
:101A2000F5500009D8A417EF8DF019EF8DF0F4EF01
:101A30008CF074C017F075C018F01200DF0E0001B2
:101A4000ED6F000EEE6FDBC0EFF0DCC0F0F0000ECB
:101A5000F36F000EF26F000EF96F000EF86FEF0ECD
:101A6000176E000E186EDDC019F0DEC01AF0ED0E14
:101A70001B6E000E1C6EE9EC8CF017C0EBF018C06A
:101A8000ECF00001F251DB25D96EF351DC21DA6E66
:101A9000000EDF6EEBC0DBF0ECC0DCF012002C6E51
:101AA00039019991050E966E000E956E000E926E9C
:101AB000770E946EF40E936E000E0001856F000E8B
:101AC000846F948E3901A9912C50D8B46AEF8DF0AF
:101AD0006CEF8DF074EF8DF02CC082F00001836B01
:101AE000390199817AEF8DF09991000E0001836F91
:0A1AF000000E826F3901A991120067
:101AFC003901A9A184EF8DF086EF8DF0AAEF8DF05E
:101B0C0099A18BEF8DF08DEF8DF0AAEF8DF0000188
:101B1C0083BF99EF8DF0835108E18205D8A099EF2E
:101B2C008DF09BEF8DF0A0EF8DF08207D8A083078E
:101B3C00A3EF8DF0BF8B39019991000E0001856FD9
:101B4C00010E846F3901A99111002CC02EF02DC00B
:101B5C002FF0B3EF8DF02C4A2D2A6000B3F0F6FF76
:101B6C006000B7F0F7FF000EF86E1F0EF76403D09D
:101B7C000800F55007D06F00DBFFE1FF6F00DFFFBF
:101B8C00E2FFE7500009D8A4CEEF8DF0D0EF8DF036
:101B9C00B1EF8DF02E502C5C2C6E2F502D582D6EDD
:101BAC001200EFEF8DF03901A3A9DFEF8DF0E1EF1B
:101BBC008DF0D9EF8DF06000B3F0F6FF6000B7F058
:101BCC00F7FF000EF86E08006F00D7FFEAFD2C4AF5
:101BDC002D2A6000B3F0F6FF6000B7F0F7FF000E9F
:101BEC00F86E0800F5500009D8A4FFEF8DF001EF56
:101BFC008EF0D9EF8DF01200010E326E200E2C18E3
:101C0C002D10D8B40CEF8EF00EEF8EF027EF8EF077
:101C1C00F70E2E6EFF0E2F6E2CC030F02DC031F053
:101C2C002E5030262F503122315009E1050E305CF8
:101C3C00D8A023EF8EF025EF8EF027EF8EF0000E5C
:101C4C00326E32C02CF02D6A12002EC030F02FC034
:101C5C0031F02CC032F02DC033F06000C3F0F6FF31
:101C6C006000C7F0F7FF304A312A000EF86E6000B2
:101C7C00CBF0D9FF6000CFF0DAFF324A332A0800EC
:101C8C006F00D7FFDFFFDF50D8A44FEF8EF051EF7E
:101C9C008EF033EF8EF01200313233413435364250
:101CAC00373839432A30234400EF3C0100395E01B8
:101CBC00003083010015AC0100B7B60000DAC90092
:101CCC000059DF0000ADF60000B9043805C5056108
:101CDC0006B90202035403AD03286E756C6C29001F
:101CEC00000E3D01EC6F000EED6F000EEE6F000E5E
:101CFC00EF6F000EF06F000EF16FB00EF26F800EF2
:101D0C00F36F000EF46F8A0EF56F000EF66F000E77
:101D1C00F76F000EF86F000EF96F000EFA6FF28B72
:101D2C00F289390193971200000E3B6E000E3A6E49
:101D3C00ABEF8EF039C02CF02D6A37C02EF038C0C6
:101D4C002FF0BAEC8AF03A4A3B2A3A503524D96E35
:101D5C003B503620DA6EDF50396E3950D8A4B9EFCB
:101D6C008EF0BBEF8EF0A0EF8EF01200272A2E32F1
:101D7C0035393C3F424447484A4B4C4D4D4D4C4BFA
:101D8C004A484744423F3C3935322E2A27231F1BF1
:101D9C001814110E0B0906050302010101010102C1
:101DAC00030506090B0E1114181B1F2332363B407A
:101DBC0044494D5155585B5D5F6162636363626179
:101DCC005F5D5B5855514D4944403B36322D2823BD
:101DDC001F1A16120E0B0806040201010101010262
:101DEC000406080B0E12161A1F23282D3FBE09EFEE
:101DFC008FF03F5006E13E04D8B007EF8FF009EFAB
:101E0C008FF017EF8FF03EC040F03FC041F0401E06
:101E1C00411E404A412A40C03EF041C03FF01BEFFA
:101E2C008FF03EC03EF03FC03FF01200000ED2BE1D
:101E3C00010E2C6ED28AD29E550ED46EAA0ED46E82
:101E4C00D490000ED76E000ED66E080ED56E550EC1
:101E5C00D46EAA0ED46ED4802CB002D0D29E01D0F7
:101E6C00D28E39018387848189811200D00E2E6E27
:101E7C00FF0E2F6E2CC030F02DC031F02E503026BE
:101E8C002F50312231500AE10A0E305CD8A051EFAC
:101E9C008FF054EF8FF0010E55EF8FF0000E2C6E7B
:101EAC002D6A12002CC02EF02DC02FF0D8902F329E
:101EBC002E32D8902F322E322E506D6E2CC02EF02A
:101ECC00030E2E16060E2F6ED8902E362F2E6AEF7E
:101EDC008FF02E506C6E12003901A3A978EF8FF0A1
:101EEC007AEF8FF072EF8FF00D0E3D01EA6F390132
:101EFC00A3A983EF8FF085EF8FF07DEF8FF00A0EA3
:101F0C003D01EA6F12002C502E026F00CCFF30F016
:101F1C006F00D0FF31F02C502F02F35031262D5092
:101F2C002E02F350312630C02CF031C02DF01200AF
:101F3C00000E3901C06F000EC16F000EC26F000E93
:101F4C00C36F000EC46F000EC56F000EC66F000E7F
:101F5C00C76F1200000EAC6E010EAE6E000EAD6EB1
:101F6C00040EAF6EAB68000EAA6E3901A495AC8E50
:101F7C0012002C6E3901A3A9C6EF8FF0C8EF8FF0B9
:101F8C00C0EF8FF06000B3F0EAFD1200A30E2D6ECF
:101F9C00570E2C6E020EE82EFED72C2EFCD72D2EB3
:101FAC00FAD700D012008C0E7E6E000E7D6E800E65
:101FBC007C6E3F015E51FC0B01095E6F1200600EDE
:101FCC003901D96F000EDB6F000EDD6F080EDF6F6D
:101FDC00000EDE6F1200800E6E6E000E6D6E000E27
:101FEC006C6E3F015F51FC0B01095F6F1200E5EC59
:101FFC008FF09EEC8FF078EC8CF0D9EC8FF0B0EC8D
:06200C008FF0120012002B
:022014001100B9
:020000040020DA
:10000000FF0FFF0FFF0FFF0FFF0FFF0FFF0FFF0F80
:020000040030CA
:0A0000008CFFFFFF9FFFFFFFFFFFD3
:00000001FF
